 gpio

 Timestamp is 4fb04cc3 (Mon May 14 12:07:31 2012)

 Preferred load address is 10000000

 Start         Length     Name                   Class
 0001:00000000 00000004H .CRT$XCA                CODE
 0001:00000004 00000004H .CRT$XCZ                CODE
 0001:00000008 00000004H .CRT$XIA                CODE
 0001:0000000c 00000004H .CRT$XIZ                CODE
 0001:00000010 00000004H .CRT$XPA                CODE
 0001:00000014 00000004H .CRT$XPZ                CODE
 0001:00000018 00000004H .CRT$XTA                CODE
 0001:0000001c 00000004H .CRT$XTZ                CODE
 0001:00000020 00001050H .rdata                  CODE
 0001:00001070 00000021H .rdata$debug            CODE
 0001:00001094 000016a8H .text                   CODE
 0001:0000273c 00000014H .xdata                  CODE
 0001:00002750 00000028H .idata$2                CODE
 0001:00002778 00000014H .idata$3                CODE
 0001:0000278c 000000c0H .idata$4                CODE
 0001:0000284c 00000130H .idata$6                CODE
 0001:00002980 000000d8H .edata                  CODE
 0002:00000000 000000c0H .idata$5                DATA
 0002:000000c0 0000044cH .data                   DATA
 0002:00000510 00000014H .bss                    DATA
 0003:00000000 000000c0H .pdata                  DATA

  Address         Publics by Value              Rva+Base       Lib:Object

 0000:00000000       ___safe_se_handler_count   00000000     <absolute>
 0000:00000000       ___safe_se_handler_table   00000000     <absolute>
 0001:00000000       __xc_a                     10001000     corelib0:crt0init.obj
 0001:00000004       __xc_z                     10001004     corelib0:crt0init.obj
 0001:00000008       __xi_a                     10001008     corelib0:crt0init.obj
 0001:0000000c       __xi_z                     1000100c     corelib0:crt0init.obj
 0001:00000010       __xp_a                     10001010     corelib0:crt0init.obj
 0001:00000014       __xp_z                     10001014     corelib0:crt0init.obj
 0001:00000018       __xt_a                     10001018     corelib0:crt0init.obj
 0001:0000001c       __xt_z                     1000101c     corelib0:crt0init.obj
 0001:00001040       ??_C@_1M@KOOMHKJP@?$AAP?$AAo?$AAr?$AAt?$AA1?$AA?$AA@ 10002040     Gpio.obj
 0001:0000104c       ??_C@_1M@LMFJNFHB@?$AAP?$AAo?$AAr?$AAt?$AA2?$AA?$AA@ 1000204c     Gpio.obj
 0001:00001058       ??_C@_1M@EOFLCBE@?$AAP?$AAo?$AAr?$AAt?$AA3?$AA?$AA@ 10002058     Gpio.obj
 0001:00001064       ??_C@_1M@JJDCIKKN@?$AAP?$AAo?$AAr?$AAt?$AA4?$AA?$AA@ 10002064     Gpio.obj
 0001:00001094       DllMain                    10002094 f   Gpio.obj
 0001:000010ac       ?GpioIntrThread@@YAKPAX@Z  100020ac f   Gpio.obj
 0001:00001110       ?CleanInterruptHandler@@YAXPAUINTR_INFO@@@Z 10002110 f   Gpio.obj
 0001:000011dc       ?SetupInterruptHandler@@YAHPAUINTR_INFO@@@Z 100021dc f   Gpio.obj
 0001:0000132c       ?Deinit@@YAHPAUDRIVER_INFO@@@Z 1000232c f   Gpio.obj
 0001:00001374       ?Open@@YAPAUOPEN_INFO@@PAUDRIVER_INFO@@KK@Z 10002374 f   Gpio.obj
 0001:000013e8       ?Close@@YAHPAUOPEN_INFO@@@Z 100023e8 f   Gpio.obj
 0001:0000142c       ?Read@@YAKPAUOPEN_INFO@@PAEK@Z 1000242c f   Gpio.obj
 0001:00001490       ?Write@@YAKPAUOPEN_INFO@@PAEK@Z 10002490 f   Gpio.obj
 0001:000014f4       ?Seek@@YAKPAUOPEN_INFO@@JK@Z 100024f4 f   Gpio.obj
 0001:00001558       ?PowerUp@@YAHPAUDRIVER_INFO@@@Z 10002558 f   Gpio.obj
 0001:00001560       ?PowerDown@@YAHPAUDRIVER_INFO@@@Z 10002560 f   Gpio.obj
 0001:00001874       ?Init@@YAPAUDRIVER_INFO@@PAX@Z 10002874 f   Gpio.obj
 0001:00001bd4       ?IOControl@@YAHPAUOPEN_INFO@@KPAEK1KPAK@Z 10002bd4 f   Gpio.obj
 0001:0000214c       EventModify                1000314c f   coredll:COREDLL.dll
 0001:0000215c       DisableThreadLibraryCalls  1000315c f   coredll:COREDLL.dll
 0001:0000216c       WaitForSingleObject        1000316c f   coredll:COREDLL.dll
 0001:0000217c       InterruptDone              1000317c f   coredll:COREDLL.dll
 0001:0000218c       CeSetThreadPriority        1000318c f   coredll:COREDLL.dll
 0001:0000219c       CloseHandle                1000319c f   coredll:COREDLL.dll
 0001:000021ac       TerminateThread            100031ac f   coredll:COREDLL.dll
 0001:000021bc       InterruptDisable           100031bc f   coredll:COREDLL.dll
 0001:000021cc       KernelIoControl            100031cc f   coredll:COREDLL.dll
 0001:000021dc       CreateThread               100031dc f   coredll:COREDLL.dll
 0001:000021ec       InterruptInitialize        100031ec f   coredll:COREDLL.dll
 0001:000021fc       CreateEventW               100031fc f   coredll:COREDLL.dll
 0001:0000220c       DeleteCriticalSection      1000320c f   coredll:COREDLL.dll
 0001:0000221c       SetLastError               1000321c f   coredll:COREDLL.dll
 0001:0000222c       RegCloseKey                1000322c f   coredll:COREDLL.dll
 0001:0000223c       RegQueryValueExW           1000323c f   coredll:COREDLL.dll
 0001:0000224c       OpenDeviceKey              1000324c f   coredll:COREDLL.dll
 0001:0000225c       InitializeCriticalSection  1000325c f   coredll:COREDLL.dll
 0001:0000226c       LeaveCriticalSection       1000326c f   coredll:COREDLL.dll
 0001:0000227c       GetLastError               1000327c f   coredll:COREDLL.dll
 0001:0000228c       EnterCriticalSection       1000328c f   coredll:COREDLL.dll
 0001:0000229c       DDKGpioClearIntrPin        1000329c f   cspddk:CSPDDK.dll
 0001:000022ac       DDKGpioGetConfig           100032ac f   cspddk:CSPDDK.dll
 0001:000022bc       DDKIomuxGetPadConfigPort   100032bc f   cspddk:CSPDDK.dll
 0001:000022cc       DDKIomuxGetPinMux          100032cc f   cspddk:CSPDDK.dll
 0001:000022dc       DDKGpioSetConfig           100032dc f   cspddk:CSPDDK.dll
 0001:000022ec       DDKIomuxSetPadConfigPort   100032ec f   cspddk:CSPDDK.dll
 0001:000022fc       DDKIomuxSetPinMux          100032fc f   cspddk:CSPDDK.dll
 0001:0000230c       DDKGpioReadIntr            1000330c f   cspddk:CSPDDK.dll
 0001:0000231c       DDKGpioReadIntrPin         1000331c f   cspddk:CSPDDK.dll
 0001:0000232c       DDKGpioReadDataPin         1000332c f   cspddk:CSPDDK.dll
 0001:0000233c       DDKGpioWriteDataPin        1000333c f   cspddk:CSPDDK.dll
 0001:0000234c       DDKGpioReadData            1000334c f   cspddk:CSPDDK.dll
 0001:0000235c       DDKGpioWriteData           1000335c f   cspddk:CSPDDK.dll
 0001:00002470       _DllMainCRTStartup         10003470 f   corelib0:pegdmain.obj
 0001:0000259c       _cexit                     1000359c f   corelib0:cexit.obj
 0001:000025b8       _initterm                  100035b8 f   corelib0:crt0dat.obj
 0001:000025ec       _cinit                     100035ec f   corelib0:crt0dat.obj
 0001:00002620       __security_init_cookie     10003620 f   corelib0:seccinit.obj
 0001:0000267c       ??3@YAXPAX@Z               1000367c f   corelib1:COREDLL.dll
 0001:0000268c       free                       1000368c f   corelib1:COREDLL.dll
 0001:0000269c       ??2@YAPAXI@Z               1000369c f   corelib1:COREDLL.dll
 0001:000026ac       memset                     100036ac f   corelib1:COREDLL.dll
 0001:000026bc       _wcsdup                    100036bc f   corelib1:COREDLL.dll
 0001:000026cc       wcscpy                     100036cc f   corelib1:COREDLL.dll
 0001:000026dc       memcpy                     100036dc f   corelib1:COREDLL.dll
 0001:000026ec       _XcptFilter                100036ec f   corelib1:COREDLL.dll
 0001:000026fc       __C_specific_handler       100036fc f   corelib1:COREDLL.dll
 0001:0000270c       __security_gen_cookie2     1000370c f   corelib1:COREDLL.dll
 0001:0000271c       InterlockedExchange        1000371c f   coredll:COREDLL.dll
 0001:0000272c       TerminateProcess           1000372c f   coredll:COREDLL.dll
 0001:00002750       __IMPORT_DESCRIPTOR_COREDLL 10003750     coredll:COREDLL.dll
 0001:00002764       __IMPORT_DESCRIPTOR_CSPDDK 10003764     cspddk:CSPDDK.dll
 0001:00002778       __NULL_IMPORT_DESCRIPTOR   10003778     coredll:COREDLL.dll
 0002:00000000       __imp_EventModify          10004000     coredll:COREDLL.dll
 0002:00000004       __imp_DisableThreadLibraryCalls 10004004     coredll:COREDLL.dll
 0002:00000008       __imp_WaitForSingleObject  10004008     coredll:COREDLL.dll
 0002:0000000c       __imp_InterruptDone        1000400c     coredll:COREDLL.dll
 0002:00000010       __imp_CeSetThreadPriority  10004010     coredll:COREDLL.dll
 0002:00000014       __imp_CloseHandle          10004014     coredll:COREDLL.dll
 0002:00000018       __imp_TerminateThread      10004018     coredll:COREDLL.dll
 0002:0000001c       __imp_InterruptDisable     1000401c     coredll:COREDLL.dll
 0002:00000020       __imp_KernelIoControl      10004020     coredll:COREDLL.dll
 0002:00000024       __imp_CreateThread         10004024     coredll:COREDLL.dll
 0002:00000028       __imp_InterruptInitialize  10004028     coredll:COREDLL.dll
 0002:0000002c       __imp_CreateEventW         1000402c     coredll:COREDLL.dll
 0002:00000030       __imp_DeleteCriticalSection 10004030     coredll:COREDLL.dll
 0002:00000034       __imp_SetLastError         10004034     coredll:COREDLL.dll
 0002:00000038       __imp_RegCloseKey          10004038     coredll:COREDLL.dll
 0002:0000003c       __imp_RegQueryValueExW     1000403c     coredll:COREDLL.dll
 0002:00000040       __imp_OpenDeviceKey        10004040     coredll:COREDLL.dll
 0002:00000044       __imp_InitializeCriticalSection 10004044     coredll:COREDLL.dll
 0002:00000048       __imp_LeaveCriticalSection 10004048     coredll:COREDLL.dll
 0002:0000004c       __imp_GetLastError         1000404c     coredll:COREDLL.dll
 0002:00000050       __imp_EnterCriticalSection 10004050     coredll:COREDLL.dll
 0002:00000054       __imp_TerminateProcess     10004054     coredll:COREDLL.dll
 0002:00000058       __imp_InterlockedExchange  10004058     coredll:COREDLL.dll
 0002:0000005c       __imp___security_gen_cookie2 1000405c     corelib1:COREDLL.dll
 0002:00000060       __imp___C_specific_handler 10004060     corelib1:COREDLL.dll
 0002:00000064       __imp__XcptFilter          10004064     corelib1:COREDLL.dll
 0002:00000068       __imp_memcpy               10004068     corelib1:COREDLL.dll
 0002:0000006c       __imp_wcscpy               1000406c     corelib1:COREDLL.dll
 0002:00000070       __imp__wcsdup              10004070     corelib1:COREDLL.dll
 0002:00000074       __imp_memset               10004074     corelib1:COREDLL.dll
 0002:00000078       __imp_??2@YAPAXI@Z         10004078     corelib1:COREDLL.dll
 0002:0000007c       __imp_??3@YAXPAX@Z         1000407c     corelib1:COREDLL.dll
 0002:00000080       __imp_free                 10004080     corelib1:COREDLL.dll
 0002:00000084       \177COREDLL_NULL_THUNK_DATA 10004084     coredll:COREDLL.dll
 0002:00000088       __imp_DDKGpioWriteData     10004088     cspddk:CSPDDK.dll
 0002:0000008c       __imp_DDKGpioReadData      1000408c     cspddk:CSPDDK.dll
 0002:00000090       __imp_DDKGpioWriteDataPin  10004090     cspddk:CSPDDK.dll
 0002:00000094       __imp_DDKGpioReadDataPin   10004094     cspddk:CSPDDK.dll
 0002:00000098       __imp_DDKGpioReadIntrPin   10004098     cspddk:CSPDDK.dll
 0002:0000009c       __imp_DDKGpioReadIntr      1000409c     cspddk:CSPDDK.dll
 0002:000000a0       __imp_DDKIomuxSetPinMux    100040a0     cspddk:CSPDDK.dll
 0002:000000a4       __imp_DDKIomuxSetPadConfigPort 100040a4     cspddk:CSPDDK.dll
 0002:000000a8       __imp_DDKIomuxGetPinMux    100040a8     cspddk:CSPDDK.dll
 0002:000000ac       __imp_DDKIomuxGetPadConfigPort 100040ac     cspddk:CSPDDK.dll
 0002:000000b0       __imp_DDKGpioGetConfig     100040b0     cspddk:CSPDDK.dll
 0002:000000b4       __imp_DDKGpioClearIntrPin  100040b4     cspddk:CSPDDK.dll
 0002:000000b8       __imp_DDKGpioSetConfig     100040b8     cspddk:CSPDDK.dll
 0002:000000bc       \177CSPDDK_NULL_THUNK_DATA 100040bc     cspddk:CSPDDK.dll
 0002:000000c0       ?dpCurSettings@@3U_DBGPARAM@@A 100040c0     DebugZones.obj
 0002:00000504       __security_cookie          10004504     corelib0:seccinit.obj
 0002:00000508       __security_cookie_complement 10004508     corelib0:seccinit.obj
 0002:00000510       _exitflag                  10004510     corelib0:cexit.obj
 0002:00000514       __onexitend                10004514     <common>
 0002:00000518       __onexitbegin              10004518     <common>
 0002:0000051c       g_pcsExit                  1000451c     <common>
 0002:00000520       _pRawDllMain               10004520     <common>

 entry point at        0001:00002470

 Static symbols

 0001:00001568       ?GetGpioConfig@@YAXPAUGPIO_CONFIG@@@Z 10002568 f   Gpio.obj
 0001:000019bc       ?SetGpioConfig@@YAXPAUGPIO_CONFIG@@H@Z 100029bc f   Gpio.obj
 0001:00002374       _DllMainCRTStartupHelper   10003374 f   corelib0:pegdmain.obj
 0001:000024a0       doexit                     100034a0 f   corelib0:cexit.obj
